:020000040800F2
:10000000B8090020C10D0008FD050008FF05000823
:1000100003060008070600080B06000800000000A1
:100020000000000000000000000000000F060008B3
:10003000110600080000000013060008150600085D
:10004000DB0D0008DB0D0008DB0D0008DB0D0008F0
:10005000DB0D0008DB0D0008DB0D0008DB0D0008E0
:10006000DB0D0008DB0D0008DB0D0008DB0D0008D0
:10007000DB0D0008DB0D0008DB0D0008DB0D0008C0
:10008000DB0D0008DB0D0008DB0D0008DB0D0008B0
:10009000DB0D0008DB0D0008DB0D0008DB0D0008A0
:1000A000DB0D0008DB0D0008DB0D0008DB0D000890
:1000B000DB0D0008DB0D0008A1040008DB0D0008C3
:1000C000DB0D0008DB0D0008DB0D0008DB0D000870
:1000D000DB0D0008390D0008B70B0008B30C000851
:1000E000DB0D0008DB0D0008DB0D0008DB0D000850
:1000F000DB0D0008DB0D0008DB0D0008DB0D000840
:10010000DB0D0008DB0D0008DB0D0008DB0D00082F
:10011000DB0D0008DB0D0008DB0D0008DB0D00081F
:10012000DB0D0008DB0D0008DB0D0008DB0D00080F
:1001300000F002F800F03AF80AA090E8000C8244BF
:100140008344AAF10107DA4501D100F02FF8AFF29C
:10015000090EBAE80F0013F0010F18BFFB1A43F0A5
:1001600001031847242A0000442A0000103A24BF43
:1001700078C878C1FAD8520724BF30C830C144BF0C
:1001800004680C607047000000230024002500264E
:10019000103A28BF78C1FBD8520728BF30C148BFEA
:1001A0000B6070471FB51FBD10B510BD02F0A5FC58
:1001B0001146FFF7F7FF00F0CDF902F0D7FC03B4CA
:1001C000FFF7F2FF03BC00F0A7FB000030B50246CA
:1001D0000B4600210020002400BF02E0555C2C44A7
:1001E000491C9942FADBE0B2C5436D1CE8B230BD50
:1001F00008B501211C2001F08DF942F20600ADF88E
:10020000000048208DF803006946E74800F0C6FE6C
:1002100008BD10B50221E44800F053FF58B14FF477
:100220000051E14800F04DFF28B10421DE4800F004
:1002300048FF002847D1DD480078002846D101203A
:10024000DA4908700221D84800F03BFF40B901208C
:10025000D7490870D74800880F30D649088035E064
:100260004FF40051D04800F02CFF40B90120D24992
:100270000870D24800880F30D049088026E0042159
:10028000C94800F01EFF08BBCDA002F0DBFA002039
:10029000C7490870C7490880C7490870C74908801E
:1002A000012080F3138800BF00BFC748006800F436
:1002B000E060C6490843001DC3490860BFF34F8F83
:1002C00000BF00BFFEE70020B8490870142010BD31
:1002D00010B5BF4890F82F01002843D0BC4890F8D3
:1002E0002E0100283EDDBA4890F82E01962839DA12
:1002F000B74890F82E0103282AD1B54890F8980005
:10030000882825D1B24890F89900552820D1B048C6
:1003100090F89A0099281BD1A64800780002AC49B1
:1003200081F89800A3480178A94880F89910A3485B
:1003300000780002C1B2A64880F89A109F48017860
:10034000A34880F89B100421983000F028FC05E0B9
:100350009F4890F82E11983000F062FB00209C49D5
:1003600081F82F019A4890F8970000287DD000204E
:10037000974981F89700084690F89600002874DDA8
:10038000084690F8960096286FDA08460078062806
:100390006CD10846407830287CD1084680781628F1
:1003A00078D10846C078022874D10846007901281F
:1003B00070D1084690F89600411E8548FFF706FF69
:1003C000834991F89610491E814A515C884266D152
:1003D0001046007B1146C97A40EA01207D49088019
:1003E0001046807B1146497B40EA01207A4908800B
:1003F0006F480078C0B1774800886E490988401A74
:100400007649086008460068012801DA0120086082
:1004100072480088724908800846008800126C49BA
:10042000C8726F480078087363480078D8B16A488A
:1004300000886249098808446849086008460068DD
:1004400040F2C641884202DD0846644908606348BC
:100450000088644908800846008800125C49487397
:100460006048007888735A4801E018E012E090F87C
:100470009600411E5648FFF7A9FE0146544890F8E1
:100480009600401E524A1154104690F8961000F003
:1004900086FB04E04E4890F8961000F080FB10BDFB
:1004A00010B50121504802F08AF9044654B10121E7
:1004B0004D4802F08DF94D480068401C4B490860DA
:1004C000FFF7A7FE10BD1FB50121042001F02FF892
:1004D00044F61F60ADF808004720ADF80400002086
:1004E000ADF80A00ADF806003F4801F07BFA01A91B
:1004F0003D4801F04BFB01213B4801F0A3FE0122E6
:100500001146394801F0B9FE1E208DF80000022086
:100510008DF8010000208DF8020001208DF8030005
:10052000684600F072FC1FBD70B505460C4645F2EA
:10053000555002F065F9284602F065F9204602F0B0
:1005400065F902F066F902F069F970BD10B502F0C4
:1005500060F910BD4FF4A06000F052FC00F072F999
:1005600000F04AF94FF4165000F0E5F94FF4165038
:1005700000F0B7FAFFF73CFEFFF7A5FF1CA002F062
:1005800061F940F271210420FFF7CEFF0AE017481D
:100590000068322802D9002014490860FFF798FE4D
:1005A000FFF7D4FFF3E7000000100140180000201F
:1005B000080000200A000020090000200C00002094
:1005C0006B330D0A000000000CED00E00000FA059E
:1005D0002602002004000020060000201400002055
:1005E0000E00002010000020000800400000002045
:1005F0007379735F696E69740D0A0000704700BFFC
:10060000FEE700BFFEE700BFFEE700BFFEE7704762
:1006100070477047704700000CB5002001900090B3
:100620006C48006840F480306A49086000BF69483F
:10063000006800F4003000900198401C0190009880
:1006400018B90198B0F5A06FF1D16248006800F4C4
:10065000003010B10120009001E0002000900098CF
:10066000012843D15C48006840F010005A490860F6
:100670000846006820F0030008600846006840F063
:100680000200086053484068524948600846406884
:1006900048600846406840F480604860084640680A
:1006A00020F47C1048600846406840F4E810486038
:1006B0000846006840F08070086000BF4548006848
:1006C00000F000700028F9D04248406820F0030094
:1006D000404948600846406840F00200486000BF5A
:1006E0003C48406800F00C000828F9D10CBD10B55A
:1006F000FFF792FF10BD10B53648006840F00100CA
:100700003449086008464068344908403149486027
:1007100008460068324908402E49086008460068CB
:1007200020F4802008600846406820F4FE004860FD
:100730004FF41F008860FFF7DAFF4FF0006029498F
:10074000086010BD10B5002100200022214B5B681D
:1007500003F00C0121B1042906D0082928D107E0B3
:10076000214B224C236027E01F4B204C236023E0C9
:10077000184B5B6803F47010164B5B6803F480320F
:10078000022303EB904022B9194B4343174C2360DB
:100790000DE0104B5B6803F4003323B1144B43436B
:1007A000124C236003E0104B4343104C236003E0E2
:1007B0000D4B0E4C236000BF00BF064B5B68C3F3BC
:1007C00003130C4CE15C094B1B68CB40074C2360C6
:1007D00010BD000000100240002002400000FFF8A1
:1007E000FFFFF6FE08ED00E000127A001C0000207A
:1007F00000093D002000002008B50121182000F06C
:1008000089FE4FF47040ADF8000010208DF8030011
:1008100003208DF802006946084800F0BFFB4FF442
:100820006040ADF8000010208DF8030003208DF823
:1008300002006946024800F0B1FB08BD000C01400F
:100840000010014010B56FF0040000F028FB2E48A6
:1008500000682E49B0FBF1F02D4908700846007879
:1008600000EB4001C1EBC0104FF6FF7101EAC00080
:100870002849088010BD0146254A12784A434FF0A6
:10088000E0235A6100229A611A46126942F001027D
:100890001A6100BF4FF0E022106900F001021AB1A6
:1008A00000F48032002AF5D04FF0E022126922F0E5
:1008B00001024FF0E0231A6100229A61704701465D
:1008C000144A12884A434FF0E0235A6100229A6189
:1008D0001A46126942F001021A6100BF4FF0E0228D
:1008E000106900F001021AB100F48032002AF5D03C
:1008F0004FF0E022126922F001024FF0E0231A616A
:1009000000229A61704700001C00002000127A004B
:100910003000002032000020014600BF704700BFB9
:10092000FB4A128802F04002002AF9D0C2B2F84B0A
:100930001B1D1A80704710B586B00446012144F291
:10094000040000F0E7FD4FF40070ADF81400032040
:100950008DF8160018208DF8170005A9ED4800F055
:100960001DFB4FF48060ADF8140004208DF81700D3
:1009700005A9E84800F012FB25208DF800000020B2
:100980008DF8010003208DF8020001208DF803008E
:10099000684600F03AFA01940020ADF80800ADF87E
:1009A0000A00ADF80C00ADF810000C20ADF80E00F8
:1009B00001A9D74800F055FE012240F22441D44855
:1009C00000F0E7FE012240F22551D14800F0E1FE9F
:1009D0000121CF4800F0D1FE06B010BD70B504462D
:1009E00025460BE000BF4021C94800F0A1FF0028C8
:1009F000F9D015F8011BC64800F02CFF204601F085
:100A00003FFF2044A842EDD870BD00BFC04909880F
:100A100001F040010029F9D0BD49091D0880704747
:100A200010B502460B4604E012F8010BFFF7EDFF8C
:100A30005B1E002BF8DC10BD10B586B0044601210A
:100A4000880400F074FD0121082000F063FD2720D8
:100A50008DF8040000208DF805008DF806000120B7
:100A60008DF8070001A800F0D0F94FF48060ADF8D0
:100A7000000003208DF8020018208DF8030069465D
:100A8000A54800F08BFA4FF40060ADF80000042098
:100A90008DF803006946A04800F080FA0294002017
:100AA000ADF80C00ADF80E00ADF81000ADF8140074
:100AB0000C20ADF8120002A9984800F0D2FD0122E6
:100AC00040F22441954800F064FE012240F2255195
:100AD000924800F05EFE0121904800F04EFE06B004
:100AE00010BD10B586B004460121480400F01FFD7A
:100AF0000121042000F00EFD0420ADF814000320B5
:100B00008DF8160018208DF8170005A9814800F00F
:100B100045FA0820ADF8140004208DF8170005A947
:100B20007C4800F03BFA01940020ADF80800ADF8D5
:100B30000A00ADF80C00ADF810000C20ADF80E0066
:100B400001A9774800F08DFD26208DF800000020D7
:100B50008DF801008DF8020001208DF80300684631
:100B600000F053F9012240F225516D4800F011FECA
:100B7000012240F224416A4800F00BFE012168483E
:100B800000F0FBFD06B010BD00BF6549098801F00B
:100B900040010029F9D06249091D0880704710B54D
:100BA00002460B4604E012F8010BFFF7EDFF5B1E57
:100BB000002BF8DC10BD10B5002440F22551584838
:100BC00000F0CCFEA0B1564800F048FEC4B2554833
:100BD0000068952804D2544852490968445402E0F8
:100BE0000020504908604F480068401C4D4908608B
:100BF00040F224414A4800F0B1FEC0B148480088A4
:100C0000C4B24748001D0088C4B24648464902683D
:100C1000464801F054FE01204449983981F82F01DB
:100C20004048007881F82E0100203E49086010BD40
:100C30002DE9F04781460F461546984600240026C8
:100C40002946484601F00AFE0446284601F018FEEF
:100C5000204400F1010A4146504601F0FFFD0646DE
:100C600014B10EB1B44202D90020BDE8F087284685
:100C700001F006FE0444321B2146384601F064FEB2
:100C80000120F2E700BF2549098801F04001002951
:100C9000F9D02249091D0880704710B502460B465D
:100CA00004E012F8010BFFF7EDFF5B1E002BF8DCF0
:100CB00010BD10B5002440F22551184800F04EFE3A
:100CC000A0B1164800F0CAFDC4B2194800689528C2
:100CD00004D2184816490968445402E00020144917
:100CE000086013480068401C1149086040F2244124
:100CF0000A4800F033FE48B108480088C4B20748EB
:100D0000001D0088C4B200200949086010BD000021
:100D10000038014000080140000C0140004800403C
:100D2000004400404400002090010020BE0200204A
:100D3000340000206400002010B5002440F225514A
:100D40001B4800F00BFEA0B1194800F087FDC4B2AB
:100D500018480068952804D2174816490968445471
:100D600002E000201349086012480068401C114945
:100D7000086040F224410E4800F0F0FDB8B10C4884
:100D80000088C4B20A48001D0088C4B209480A4954
:100D900002680A4801F093FD0120084981F8970094
:100DA0000448007881F8960000200249086010BDD0
:100DB000003801403C000020FA00002026020020FC
:100DC0000948804709480047FEE7FEE7FEE7FEE7DF
:100DD000FEE7FEE7FEE7FEE7FEE7FEE7044805491B
:100DE000054A064B70470000F7060008310100086D
:100DF000B8030020B8090020B8050020B80500207D
:100E000031490143314A1160704770B50021002318
:100E10000F22C47804B32D4C246804F4E064C4F5B4
:100E2000E064210AC1F10403CA40447804FA03F1E2
:100E30008478144021430901254C0678A155047893
:100E400004F01F050124AC4005786D11AD0005F1DB
:100E5000E025C5F8004109E0047804F01F050124ED
:100E6000AC401C4D0678761145F8264070BD1A4AF4
:100E70000A400243154B1B1F1A60704739B1134AD1
:100E8000121D12680243114B1B1D1A6006E00F4A27
:100E9000121D126882430D4B1B1D1A6070470428F7
:100EA00008D14FF0E021096941F004014FF0E02240
:100EB000116107E04FF0E021096921F004014FF0D2
:100EC000E0221161704700000000FA050CED00E01F
:100ED00000E400E080E100E080FFFF1F10B5044661
:100EE000CC48844208D10121042000F02DFB0021D0
:100EF000042000F029FB46E0C748844208D10121C4
:100F0000082000F021FB0021082000F01DFB3AE042
:100F1000C248844208D10121102000F015FB0021B5
:100F2000102000F011FB2EE0BD48844208D10121C1
:100F3000202000F009FB0021202000F005FB22E02A
:100F4000B848844208D10121402000F0FDFA002178
:100F5000402000F0F9FA16E0B348844208D101219C
:100F6000802000F0F1FA0021802000F0EDFA0AE084
:100F7000AE48844207D10121801500F0E5FA002136
:100F8000A01500F0E1FA10BD10B50121084600F0EF
:100F9000DBFA0021012000F0D7FA10BD2DE9F04165
:100FA000024600250026002000230024002791F897
:100FB00003C00CF00F0591F803C00CF0100CBCF14D
:100FC000000F03D091F802C04CEA050591F800C06B
:100FD000BCF1000F31D0146800202BE04FF0010C61
:100FE0000CFA00F3B1F800C00CEA03069E4220D1CF
:100FF00083004FF00F0C0CFA03F7BC4305FA03FC17
:101000004CEA040491F803C0BCF1280F06D14FF05C
:10101000010C0CFA00FCC2F814C00AE091F803C0FD
:10102000BCF1480F05D14FF0010C0CFA00FCC2F8DE
:1010300010C0401C0828D1D31460B1F800C0BCF126
:10104000FF0F34DD546800202EE000F1080C4FF053
:10105000010808FA0CF3B1F800C00CEA03069E423E
:1010600021D183004FF00F0C0CFA03F7BC4305FAB3
:1010700003FC4CEA040491F803C0BCF1280F05D12D
:1010800000F1080C08FA0CF8C2F8148091F803C0BB
:10109000BCF1480F07D100F1080C4FF0010808FA25
:1010A0000CF8C2F81080401C0828CED35460BDE86C
:1010B000F0814FF6FF710180022181700421C1701F
:1010C00070470246002093680B400BB1012000E0FE
:1010D000002070470146886880B2704702460020B1
:1010E000D3680B400BB1012000E00020704701469F
:1010F000C86880B2704701617047416170470AB1AA
:10110000016100E041617047C16070474FF4803277
:101110000A43826181618261826982697047024605
:101120000020434B18684FF68073184040EA0210C5
:1011300008433F4B186070473E49C8617047F0B59F
:101140000A46002300240021002500F00046B6F1E5
:10115000004F02D1364EF16901E0354E7168C0F39F
:10116000034583B200F44016B6F5401F08D121F0C4
:1011700070612F4E766826F070662D4F7E6012E00B
:1011800000F48016B6F5801F06D1032606FA05F492
:10119000A14341F0706106E0460D360103FA06F600
:1011A000B14341F0706122B1460D360103FA06F6F3
:1011B000314300F00046B6F1004F02D11C4EF16100
:1011C00001E01B4E7160F0BD30B500228B071C0F93
:1011D0000F2303FA04F2164B08338C1053F8243013
:1011E0009343134C08348D1044F8253023468C105B
:1011F00053F824308C07240F00FA04F423430C4CDA
:1012000008348D1044F8253030BD0A49DC310860BF
:101210007047000000080140000C01400010014030
:101220000014014000180140001C01400020014052
:101230000000014000002042DF48006840F001004B
:10124000DD49086008464068DC490840DA494860E2
:1012500008460068DA490840D7490860084600682F
:1012600020F4802008600846406820F4FE004860B2
:101270004FF41F0088607047CF49096821F480311E
:10128000CD4A11601146096821F480211160B0F542
:10129000803F03D0B0F5802F0ED106E0C649096823
:1012A00041F48031C44A116007E0C349096841F440
:1012B000A021C14A116000E000BF00BF704710B517
:1012C00001460022002300204A11012A02D1BA4C13
:1012D000236806E0022A02D1B74C236A01E0B64C2B
:1012E000636A01F01F02012494401C400CB10120EC
:1012F00000E0002010BD38B500200090002400253B
:1013000000BF3120FFF7DBFF05460098401C00902E
:101310000098B0F5A06F01D0002DF2D03120FFF77A
:10132000CEFF08B1012400E00024204638BD01466C
:101330000020A14A106820F0F80040EAC1001060C7
:101340007047A04908607047024600209A4B5868D1
:1013500020F47C1042EA01031843974B5860704711
:1013600098490866704701460020934A506820F06B
:1013700003000843506070478F48406800F00C003D
:101380007047014600208C4A506820F0F000084366
:101390005060704701460020874A506820F4E060A2
:1013A00008435060704701460020834A506820F48B
:1013B000605040EAC1005060704729B17E4A527ABD
:1013C00002437D4B5A7204E07B4A527A82437A4B45
:1013D0005A7270477B49D831086070470146002037
:1013E000754A506820F4404008435060704700211F
:1013F000714A20321170704A82F82010012802D000
:1014000004280AD104E001216B4A2032117005E062
:101410000521694A2032117000E000BF00BF70470B
:101420006949086070476449096A0143624A116268
:101430007047654944390860704730B50021002283
:10144000002400235C4D6D6805F00C0121B10429D6
:1014500005D0082923D105E05C4D056022E05B4DF5
:1014600005601FE0544D6D6805F47012524D6D68B3
:1014700005F48034022505EB92421CB9544D5543C6
:1014800005600BE04C4D6D6805F400351DB1504D05
:101490005543056002E04D4D5543056002E04B4D5C
:1014A000056000BF00BF444D6D6805F0F0010909FB
:1014B000484D6B5C0568DD4045603F4D6D6805F447
:1014C000E061090A434D6B5C4568DD4085603A4D3B
:1014D0006D6805F46051C90A3E4D6B5C4568DD409E
:1014E000C560354D6D6805F44041890B3A4D6B5C24
:1014F000C568B5FBF3F5056130BD29B12E4A5269C7
:1015000002432D4B5A6104E02B4A526982432A4B15
:101510005A61704729B1284A92690243264B9A6161
:1015200004E0254A92698243234B9A61704729B1AE
:10153000214AD2690243204BDA6104E01E4AD26993
:1015400082431D4BDA61704729B11B4AD2680243BE
:10155000194BDA6004E0184AD2688243164BDA600D
:10156000704729B1144A12690243134B1A6104E00F
:10157000114A12698243104B1A617047124940396F
:10158000086070470F49C86470470B49C8717047BD
:101590000948406A40F08070074948627047014638
:1015A0000020054A92680A400AB1012000E00020AC
:1015B0007047014988727047001002400000FFF830
:1015C000FFFFF6FE000042428004424200127A0011
:1015D00000093D00500000206000002010B50446C6
:1015E000FB48844209D101218803FFF7ADFF0021A8
:1015F0004FF48040FFF7A8FF32E0F648844209D15B
:1016000001214804FFF7ADFF00214FF40030FFF740
:10161000A8FF25E0F048844209D101218804FFF7A2
:10162000A0FF00214FF48020FFF79BFF18E0EB485C
:10163000844209D10121C804FFF793FF00214FF430
:101640000020FFF78EFF0BE0E548844208D101211E
:101650000805FFF786FF00214FF48010FFF781FF98
:1016600010BD2DE9F04786B005460E460024A2467F
:1016700000BFA1460027B08900B100BF2F462C8AC9
:101680004CF6FF700440F08804432C82AC894EF67F
:10169000F3100440B088318908437189084304433A
:1016A000AC81AC8A4FF6FF400440B0890443AC8261
:1016B00001A8FFF7C2FEC648874202D1DDF810A09C
:1016C00001E0DDF80CA0A88900F4004040B10AEB6D
:1016D000CA0000EB0A1031684900B0FBF1F807E0DE
:1016E0000AEBCA0000EB0A1031688900B0FBF1F880
:1016F0006420B8FBF0F004012009642101FB10898B
:10170000A88900F4004040B1322000EBC900B0FBD2
:10171000F1F000F00700044308E0322000EB09106C
:101720006421B0FBF1F000F00F0004432C8106B0FF
:10173000BDE8F0874FF41651016000218180C1801F
:1017400001810C21418100218181704710B5024641
:101750000020108A4FF2FF0318400B884C88234367
:101760008C882343CC8823431843108210BD00216A
:10177000018041808180C180704721B1828942F41B
:101780000052828104E082894DF6FF731A40828103
:101790007047F0B50346002400260025002040F6DF
:1017A0006A17B94200D100BF1846C1F3421401F0D4
:1017B0001F06012707FA06F5012C01D10C3004E0C1
:1017C000022C01D1103000E014301AB107682F4309
:1017D000076002E00768AF430760F0BD1AB1838A73
:1017E0000B43838202E0838A8B4383827047028AA1
:1017F0004FF6F0731A400282028A0A43028270474F
:1018000082894FF2FF731A40828182890A43828162
:10181000704721B1828942F00202828104E082890C
:101820004FF6FD731A4082817047028A4FF6DF73CC
:101830001A400282028A0A430282704721B1028A58
:1018400042F48042028204E0028A4BF6FF731A409F
:1018500002827047C1F3080282807047014688887F
:10186000C0F308007047818941F001018181704710
:10187000028BD2B20283028B42EA012202837047BA
:10188000028B02F47F420283028B0A430283704779
:1018900021B1828A42F02002828204E0828A4FF6DD
:1018A000DF731A408282704721B1828A42F01002AF
:1018B000828204E0828A4FF6EF731A408282704778
:1018C00021B1828A42F00802828204E0828A4FF6C5
:1018D000F7731A408282704721B1828942F4004234
:1018E000828103E08289C2F30E028281704721B1B6
:1018F000828A42F40062828204E0828A4FF2FF739D
:101900001A4082827047828A4FF6FB731A408282A5
:10191000828A0A438282704721B1828A42F002029F
:10192000828204E0828A4FF6FD731A4082827047F9
:1019300002460020B1F5007F00D100BF13880B40A4
:101940000BB1012000E00020704701F40072B2F5F5
:10195000007F00D100BFCA430280704770B50246C5
:10196000002400230025002040F66A16B14200D171
:1019700000BFC1F3421501F01F03012606FA03F36D
:10198000012D02D19689334006E0022D02D1168A3C
:10199000334001E0968A33400C12012606FA04F423
:1019A0001688344013B10CB1012000E0002070BD56
:1019B00010B50022002340F66A14A14200D100BFF6
:1019C0000A1201249440A3B2DC43048010BD00003D
:1019D000003801400044004000480040004C0040F6
:1019E0000050004010B50446FE48844208D1012151
:1019F000C014FFF7A9FD0021E014FFF7A5FDC4E026
:101A0000B4F1804F08D101210846FFF7AAFD00215B
:101A10000120FFF7A6FDB8E0F348844208D1012178
:101A20000220FFF79EFD00210220FFF79AFDACE0A7
:101A3000EE48844208D101210420FFF792FD0021E5
:101A40000420FFF78EFDA0E0E948844208D101217F
:101A50000820FFF786FD00210820FFF782FD94E0B3
:101A6000E448844208D101211020FFF77AFD0021CB
:101A70001020FFF776FD88E0DF48844208D101217D
:101A80002020FFF76EFD00212020FFF76AFD7CE09B
:101A9000DA48844208D101214014FFF755FD0021A6
:101AA0006014FFF751FD70E0D548844209D101214F
:101AB000C804FFF749FD00214FF40020FFF744FD63
:101AC00063E0D048844209D101210805FFF73CFDBD
:101AD00000214FF48010FFF737FD56E0CA488442DA
:101AE00009D101214805FFF72FFD00214FF4001017
:101AF000FFF72AFD49E0C548844208D10121402072
:101B0000FFF72FFD00214020FFF72BFD3DE0C048EF
:101B1000844208D101218020FFF723FD002180208D
:101B2000FFF71FFD31E0BB48844208D10121801539
:101B3000FFF717FD0021A015FFF713FD25E0B648BC
:101B4000844209D101210804FFF7FEFC00214FF473
:101B50008030FFF7F9FC18E0B048844209D1012138
:101B60004804FFF7F1FC00214FF40030FFF7ECFCD4
:101B70000BE0AB48844208D101218804FFF7E4FC64
:101B800000214FF48020FFF7DFFC10BD0022028807
:101B9000944B98420ED0994B98420BD0B0F1804FA5
:101BA00008D0914B984205D0904B984202D0904B70
:101BB000984204D14FF68F731A404B881A438D4BCD
:101BC000984207D08C4B984204D04FF6FF431A40FE
:101BD000CB881A4302808B8883850B880385814BD1
:101BE00098420BD0854B984208D08B4B984205D039
:101BF0008A4B984202D08A4B984201D10B7A0386D5
:101C000001238382704770B5002400220023058CD5
:101C10004FF6FE7635400584028C8388048B4FF6A0
:101C20008F752C40B51E2C400D882C43751E2A4004
:101C30000D892A434D882A436A4DA8420BD06F4D27
:101C4000A84208D0744DA84205D0744DA84202D0D5
:101C5000734DA84213D14FF6F7752A404D892A4398
:101C60004FF6FB752A408D882A434FF6FF652B40BF
:101C70004FF6FF552B408D892B43CD892B43838015
:101C80000483CD888586028470BD70B5002400224F
:101C90000023058C4FF6EF7635400584028C83884F
:101CA000048B48F6FF752C404FF6FF452C400D88FD
:101CB0004FF6FF7606EA05252C434FF6DF752A40DE
:101CC0000D8906EA05152A434D8806EA05152A43BB
:101CD000444DA84202D0494DA8421DD14FF67F7510
:101CE0002A404D894FF6FF7606EA05152A434FF63E
:101CF000BF752A408D8806EA05152A434FF6FF3541
:101D00002B404FF2FF752B408D8906EA85052B434A
:101D1000CD8906EA85052B4383800483CD8805871A
:101D2000028470BD70B5002400220023058C4FF69C
:101D3000FF6635400584028C8388848B4FF68F754F
:101D40002C404FF6FC752C400D882C434FF6FF5568
:101D50002A400D894FF6FF7606EA05252A434D886D
:101D600006EA05252A431F4DA84202D0234DA8426A
:101D70001DD14FF2FF752A404D894FF6FF7606EAD6
:101D800005252A434FF6FF352A408D8806EA0525AA
:101D90002A434EF6FF752B404DF6FF752B408D897B
:101DA00006EA05152B43CD8906EA05152B438380EA
:101DB0008483CD888587028470BD70B5002200239E
:101DC0000024058C4EF6FF7635400584038C84880C
:101DD000828B48F6FF752A404FF6FF452A400D8852
:101DE00020E00000002C01400004004000080040FA
:101DF000000C00400010004000140040003401407E
:101E0000004C0140005001400054014000180040C7
:101E1000001C004000200040004001400044014000
:101E2000004801404FF6FF7606EA05252A434DF6A5
:101E3000FF752B400D8906EA05352B434D8806EAD0
:101E400005352B43FA4DA84202D0FA4DA84208D1DD
:101E50004BF6FF752C408D894FF6FF7606EA851507
:101E60002C4384808283CD88A0F84050038470BDC9
:101E7000828B4FF2FF331A408283828B4FF6FF73BF
:101E800003EA01231A4382837047F0B50C461546D6
:101E9000002200210026078C4EF6FF7C07EA0C0783
:101EA0000784828B018C4FF6FF7707EA043640F6F1
:101EB000FF473A404FF6FF7707EA05273A434FF6C8
:101EC000FF7707EA03373A43D94FB8420ED0D94FCC
:101ED000B8420BD0B0F1804F08D0D74FB84205D0F0
:101EE000D64FB84202D0D64FB84206D14DF6FF7752
:101EF000394046F48057394305E047F6FF573940EB
:101F000044F48057394382830184F0BD828B4FF6BD
:101F1000F3731A408283828B0A4382837047F0B541
:101F20000C461546002200210026078C4FF6FF6C58
:101F300007EA0C070784828B018C4FF6FF7707EACC
:101F400004264FF60C773A404FF6FF7707EA03175F
:101F50002F433A43B64FB8420ED0B64FB8420BD0DB
:101F6000B0F1804F08D0B44FB84205D0B34FB8425B
:101F700002D0B34FB84206D14FF6FF57394046F46E
:101F80008077394305E04FF2FF57394044F48077BA
:101F9000394382830184F0BD028B4FF2FF331A4034
:101FA0000283028B4FF6FF7303EA01231A43028375
:101FB0007047F0B50C461546002200210026078C1C
:101FC0004FF6EF7C07EA0C070784028B018C4FF673
:101FD000FF7707EA041640F6FF473A404FF6FF77CF
:101FE00007EA03373A434FF6FF7707EA05273A43F4
:101FF0008F4FB8420ED08F4FB8420BD0B0F1804F08
:1020000008D08D4FB84205D08C4FB84202D08C4FCB
:10201000B84206D14FF6DF77394046F01007394312
:1020200005E04FF65F77394044F0100739430283EB
:102030000184F0BD028B4FF6F3731A400283028BCA
:102040000A4302837047F0B50C4615460022002172
:10205000068C4FF6FE773E400684028B018C4FF6CD
:102060000C7632407E1C06EA03162E433243704E35
:10207000B0420ED06F4EB0420BD0B0F1804F08D0BE
:102080006D4EB04205D06D4EB04202D06C4EB042A3
:1020900006D14FF6FD76314044F00106314305E0AC
:1020A0004FF6F576314044F0010631430283018456
:1020B000F0BD70B505460C465D4885420ED05D48C2
:1020C00085420BD0B5F1804F08D05B48854205D0E2
:1020D0005A48854202D05A48854200D100E000BFEC
:1020E000208850B92389A28861882846FFF7ABFF72
:1020F000E1882846FFF79EFF25E0208804280AD1C2
:102100002389A28861882846FFF753FFE188284683
:10211000FFF742FF17E0208808280AD12389A28808
:1021200061882846FFF7FBFEE1882846FFF7EEFEB0
:1021300009E02389A28861882846FFF7A6FEE18886
:102140002846FFF795FE70BD2DE9F04105460C4687
:1021500000260127608808B9022600E00026A08832
:10216000012801D1022700E001272088A0B9238996
:10217000A28861882846FFF766FFE1882846FFF7B6
:1021800059FF23893A4631462846FFF712FFE18876
:102190002846FFF701FF13E02389A28861882846BB
:1021A000FFF707FFE1882846FFF7F6FE23893A4646
:1021B00031462846FFF747FFE1882846FFF73AFFF8
:1021C000BDE8F0810A884B881A438B881A43CB8874
:1021D0001A430B891A434B891A438B891A43A0F877
:1021E000442070474FF6FF71818000210180C1803B
:1021F0004180017270470021018041808180C1804F
:10220000018141818181C18170470021018041802C
:10221000012181800021C18001817047002101805E
:1022200041808180C18001814181818170470000AE
:10223000002C014000340140000400400008004030
:10224000000C004021B1028842F00102028004E04B
:1022500002884FF6FE731A400280704731B1B0F821
:10226000442042F40042A0F8442005E0B0F84420A5
:10227000C2F30E02A0F8442070471AB183890B43C1
:10228000838102E083898B43838170478182704719
:1022900041EA0203A0F8483070471AB183890B4322
:1022A000838102E083898B438381704701894FF6E4
:1022B000F8721140018170470A46002101894FF6EA
:1022C0008F73194011430181704730B504460D46A4
:1022D00029462046FFF7F0FF208940F007002081C3
:1022E00030BD2DE9F04104460D4616461F46602DCF
:1022F00006D13B46012231462046FFF75AFE05E053
:102300003B46012231462046FFF79DFE29462046E6
:10231000FFF7D2FF208940F007002081BDE8F0815F
:1023200030B50C4600210189C9B24FF6FF7505EAA8
:102330000325154325432943018130BD2DE9F04193
:1023400005460E4617469846002443463A4631460F
:102350002846FFF7E5FF2C894FF6F870044044F05B
:1023600007044FF68F70044044F070042C81BDE8E0
:10237000F081F0B504460D4616461F463B463246F0
:1023800029462046FFF7CCFF208940F48040208179
:10239000F0BD0185828270470A46002101884FF610
:1023A0008F731940114301807047F0B50C461546F4
:1023B0001E460021002200230189028B038C4FF668
:1023C000F877394021434FF6FC473A4040F2011775
:1023D0003A434FF6DD773B404FF6FF7707EA0617A3
:1023E0002F433B43018102830384F0BD0A46002151
:1023F000018B4FF68F7319401143018370470A46D2
:102400000021018B48F6FF7319404FF6FF7303EA72
:1024100002231943018370470A460021818B4FF63E
:102420008F7319401143818370470A460021818BC5
:1024300048F6FF7319404FF6FF7303EA022319436E
:102440008183704721B1028842F08002028004E05B
:1024500002884FF67F731A400280704721B182884C
:1024600042F00402828004E082884FF6FB731A4037
:102470008280704721B1828842F00802828004E0A5
:1024800082884FF6F7731A408280704721B18288A4
:1024900042F00102828004E082884FF6FE731A4007
:1024A000828070470A460021018B4FF6F77319406E
:1024B0001143018370470A460021018B4FF2FF73DD
:1024C00019404FF6FF7303EA022319430183704753
:1024D0000A460021818B4FF6F7731940114381831F
:1024E00070470A460021818B4FF2FF7319404FF667
:1024F000FF7303EA02231943818370470A460021D0
:10250000018B4FF6FB7319401143018370470A4654
:102510000021018B4FF6FF3319404FF6FF7303EA9A
:1025200002231943018370470A460021818B4FF62D
:10253000FB7319401143818370470A460021818B48
:102540004FF6FF3319404FF6FF7303EA0223194396
:10255000818370470A460021018B4FF67F73194033
:102560001143018370470A460021018BC1F30E011C
:102570004FF6FF7303EA02231943018370470A46AB
:102580000021818B4FF67F7319401143818370477F
:102590000A460021818BC1F30E014FF6FF7303EA57
:1025A00002231943818370470A460021018C4FF6AC
:1025B000FD7319401143018470470A460021018CC4
:1025C0004FF6F77319401143018470470A46002102
:1025D000018C4FF6DF7319404FF6FF7303EA0213C5
:1025E0001943018470470A460021018C4FF67F731E
:1025F00019404FF6FF7303EA021319430184704731
:102600000A460021018C4FF6FF5319404FF6FF7325
:1026100003EA02231943018470470A460021018C12
:102620004FF2FF7319404FF6FF7303EA0223194379
:10263000018470470A460021018C4DF6FF73194052
:102640004FF6FF7303EA023319430184704730B534
:10265000002301248C40A3B2048C9C430484048C8A
:1026600002FA01F5ADB22C43048430BD30B500232D
:1026700004248C40A3B2048C9C430484048C02FA8E
:1026800001F5ADB22C43048430BD70B50346002083
:1026900000241846183001258D40ACB21D8CA5438E
:1026A0001D8409B1082909D100EB6100056825F0F6
:1026B000700505600568154305600EE00D1FC5F344
:1026C0004E052844056825F4E045056005684FF689
:1026D000FF7606EA02263543056070BD21B1028807
:1026E00042F00202028004E002884FF6FD731A40B5
:1026F0000280704721B1028842F00402028004E0A7
:1027000002884FF6FB731A400280704721B182881D
:1027100042F08002828004E082884FF67F731A4084
:102720008280704702884FF6F7731A400280028851
:102730000A430280704782884FF68F731A40828066
:1027400082880A438280704702894FF6F8731A40E4
:10275000028102890A430281704702894FF67F7322
:102760001A40028102890A430281704781847047BE
:1027700081857047818670470187704781877047E0
:10278000A0F84010704702884FF6FF431A400280BD
:1027900002880A43028070470146888E70470146CE
:1027A000088F70470146888F70470146B1F8400096
:1027B00070470146888C70470146088D7047024675
:1027C0000020138A0B400BB1012000E0002070476D
:1027D000CA430282704730B502460020002300241D
:1027E000158A05EA0103958905EA010413B10CB1C4
:1027F000012000E0002030BDCA4302827047000083
:102800000E49086070470D49486070470B49886061
:1028100070474AF6AA200949086070474CF6CC4038
:1028200006490860704701460020044AD2680A4001
:102830000AB1012000E00020704700000030004095
:10284000704700000FB4044910B503AA029800F0C5
:10285000ABF810BC5DF814FB4C00002030B5054609
:102860000B462A4613F8014B12F8010B08B1A0429F
:10287000F8D01CB1002802D06D1CF1E7284630BD0D
:1028800010B5431C02E010F8011B71B18107FAD1A9
:102890004FF0013202C88C1A8C4314EAC211F9D0ED
:1028A000C01A0A0603D0C01E10BDC01A10BD0A040B
:1028B00001D0801E10BD0902FCD0401E10BD032AAD
:1028C00040F2308010F0030C00F0158011F8013B4D
:1028D000BCF1020F624498BF11F801CB00F8013B34
:1028E00038BF11F8013BA2F1040298BF00F801CBF8
:1028F00038BF00F8013B11F0030300F06780083A8D
:10290000C0F0088051F8043B083A51F804CBA0E825
:102910000810F5E7121D5CBF51F8043B40F8043B7A
:10292000AFF30080D20724BF11F8013B11F801CBAF
:1029300048BF11F8012B24BF00F8013B00F801CB80
:1029400048BF00F8012B704710B5044610F0030F84
:1029500008BF11F0030F40F015804FF0013E121F29
:10296000C0F20E8051F8043BA3EB0E0C2CEA030CD2
:102970001CEACE1C08BF40F8043BF0D0A1F10401D2
:1029800002F10402521E08DB11F8013B002B00F893
:10299000013BF7D1114600F04BF8204610BD7047BF
:1029A0007047704770470000074B70B50D467B4479
:1029B00000F065F80446284600F074F810B14FF0B6
:1029C000FF3070BD204670BD6DDFFFFF10B5203AAF
:1029D000C0F00B80B1E81850203AA0E81850B1E8D8
:1029E0001850A0E81850BFF4F5AF5FEA027C24BF8E
:1029F000B1E81850A0E8185044BF18C918C0BDE885
:102A000010405FEA827C24BF51F8043B40F8043B4D
:102A100008BF7047D20728BF31F8023B48BF11F802
:102A2000012B28BF20F8023B48BF00F8012B70475C
:102A30004FF000020429C0F0128010F0030C00F0E7
:102A40003780CCF1040CBCF1020F18BF00F8012B49
:102A5000A8BF20F8022BA1EB0C0100F029B85FEA17
:102A6000C17C24BF00F8012B00F8012B48BF00F8FF
:102A7000012B704701694A1C02610878704700B554
:102A80008FB0CDE901310021059105497944CDE9A7
:102A900003101146684600F055F80FB000BD000065
:102AA000E5FFFFFF007B00F0800070474FF0000261
:102AB00000B5134694469646203922BFA0E80C5034
:102AC000A0E80C50B1F12001BFF4F7AF090728BF0F
:102AD000A0E80C5048BF0CC05DF804EB890028BF8B
:102AE00040F8042B08BF704748BF20F8022B11F0B4
:102AF000804F18BF00F8012B7047754600F040F872
:102B0000AE4605006946534620F00700854618B0DA
:102B100020B5FEF763F9BDE820404FF000064FF006
:102B200000074FF000084FF0000B21F00701AC4602
:102B3000ACE8C009ACE8C009ACE8C009ACE8C00921
:102B40008D4670472DE9F04106460024D6E9017014
:102B5000F5688046304603E04146B847641C30467D
:102B6000A8470028F8D12046BDE8F08110B50446FA
:102B7000AFF300802046BDE81040FDF720BB000009
:102B80000048704758030020A82B000800000020D0
:102B9000640000006C0100080C2C00086400002098
:102BA0005409000088010008000000000000000037
:102BB0000000000000000000000000000000000015
:102BC0000000000000A24A04000000000000000015
:102BD00001020304060708090000000000000000CD
:102BE00000000000000000000000000000000000E5
:102BF00000000000000000000000000001020304CB
:0C2C00000102030406070809020406088C
:0400000508000131BD
:00000001FF
